:1000000000308A0004280000FF238316900000308F
:100010008A005E2B0A108A100A1182073F340634C8
:100020005B344F3466346D347D3407347F346F3441
:100030000034633463345C345C34AD08031D23281E
:10004000AE080319442883160710831207140130E1
:10005000AF002F082C02031C33282D080319AE0310
:10006000AD03AF0A29288316071083120710013049
:10007000AF002F082C02031C43282D080319AE03E0
:10008000AD03AF0A39281D2800342C082D040319AC
:1000900056280130AE002E08323C031C5128AE0A0F
:1000A0004B282C080319AD03AC03452800342C0859
:1000B0000A20D800A0002D080A20D800A10083162D
:1000C00005108312051083168510831285100130E8
:1000D000AE002E08103C031C8A2821308400000842
:1000E0008039003A031D7928831605118312051102
:1000F0007D2883160511831205150310A00DA10D8F
:10010000831605108312051483160510831205103B
:10011000AE0A6928831685108312851400340130D5
:10012000A300A401A601A701A801A21483168515A6
:10013000831285193D298316071583120719A228F2
:100140000130AB008316871483128718A828AB01EF
:100150008316071500308312071D0130AC0083168B
:10016000871400308312871C01302C04003A0319D5
:10017000E228221CC0282908A6002A08A70022106D
:10018000A4011E30A300A60AA70A0A30AC00AE01E3
:100190006430AD001D2026080F39073C031DD2280E
:1001A0000130A60027080F39073C031DD92801306C
:1001B000A7002408AD002308AC0045202830A80083
:1001C000A2141929A80803190F2928080F3C03189D
:1001D000EE280630A3070318A40AF2281430A30758
:1001E0000318A40AA803A60AA70A0A30AC00AE01A5
:1001F0006430AD001D2026080F39073C031D02297D
:100200000130A60027080F39073C031D09290130DA
:10021000A7002408AD002308AC0045201929A21C22
:1002200017290A30AC00AE016430AD001D20221445
:10023000A210221C2B29A90A29080F39073C031DEB
:100240002B290130A900AA0A2A080F39073C031DEF
:100250002B290130AA00AB08031D37290A30A7005B
:100260002608AC002708AD005720A7013C29260826
:10027000AC002708AD0057209628702BA601A401DA
:100280000130A300A701A214831687168312871AD0
:10029000C1298316871400308312871C0130AC00FB
:1002A0008316071500308312071D01302C04003A15
:1002B00003197829221C5F292808A6002210A4010E
:1002C0001E30A300A60A0A30AC00AE016430AD00B7
:1002D0001D2026080F39023C031D6F29A6012408A2
:1002E000AD002308AC0045202830A700A214A629A1
:1002F000A70803199C2927080F3C031884290630F6
:10030000A3070318A40A88291430A3070318A40A12
:10031000A703A60A0A30AC00AE016430AD001D2070
:1003200026080F39023C031D9629A6012408AD00BA
:100330002308AC004520A629A21CA4290A30AC0041
:10034000AE016430AD001D202214A210A80A2808B6
:100350000F39023C031DAD29A80126080F39003AC8
:10036000031DB7290C30AA000B30AB00BB290E309F
:10037000AA000D30AB002A08AC002B08AD005720B6
:100380004429762BA201A301831607168312071AAC
:10039000032A8316071583120719DA29A20A2208ED
:1003A0000A3C031DDA29A201A30A23080A3C031D03
:1003B000DA29A3018316071583120719E429AD0171
:1003C0006430AC004520DA2983168714831287181D
:1003D000F329A203220FF3290930A200A303230F5C
:1003E000F3290930A3008316871483128718FD2987
:1003F000AD016430AC004520F3292208AC0023088D
:10040000AD005720C4297C2B22102215A301A40182
:10041000A501A60183168715831287195D2B221C5F
:10042000362AA303230F1B2A0930A300A403240F99
:100430001B2A0930A400A308031D362AA408031DA3
:10044000362A83160512831205122308AC002408ED
:10045000AD0057200E30AC00AE015030AD001D2075
:100460002215221083160512831205162308AC00EC
:100470002408AD005720A801A7012808AC3C031CA4
:100480005C2B031D472A2708A83C031C5C2B831602
:100490008714831287186F2AA508031D522AA608FD
:1004A0000319612A221D592A2508A3002608A40041
:1004B00022110130A2060A30AC00AE01C830AD00F6
:1004C0001D20AD010A30AC0045208316871483122D
:1004D00087186F2AAD016430AC004520652A2218C8
:1004E0004B2BA21CE02AAA01A901AA08031DDE2A9F
:1004F0002908643C031CDE2A83168714831287189C
:10050000A42AA508031D872AA6080319962A221DD6
:100510008E2A2508A3002608A40022110130A20675
:100520000A30AC00AE01C830AD001D20AD010A306C
:10053000AC0045208316871483128718A42AAD01C6
:100540006430AC0045209A2A221DCD2A8316071557
:1005500083120719CD2AA50A25080A3C031DB72ACC
:10056000A501A60A26080A3C031DB72AA601A80170
:10057000A7010A30AC00AE01C830AD001D20AD01AE
:100580000A30AC0045208316071583120719CD2ABF
:10059000AD016430AC004520C32A221DD52A2508B0
:1005A000AC002608AD005720DA2A2308AC00240846
:1005B000AD005720A90A0319AA0A752AA2104B2BCD
:1005C000AA01A901AA08031D4A2B2908643C031C9F
:1005D0004A2B8316871483128718112BA508031D35
:1005E000F42AA6080319032B221DFB2A2508A300C1
:1005F0002608A40022110130A2060A30AC00AE0188
:10060000C830AD001D20AD010A30AC004520831676
:10061000871483128718112BAD016430AC0045207C
:10062000072B221D3A2B83160715831207193A2B25
:10063000A50A25080A3C031D242BA501A60A2608A5
:100640000A3C031D242BA601A801A7010A30AC0017
:10065000AE01C830AD001D20AD010A30AC00452010
:1006600083160715831207193A2BAD016430AC00CD
:100670004520302B221C422B2308AC002408AD005F
:100680005720462B0A30AC00AD005720A90A0319A9
:10069000AA0AE22AA2142218522B83168715831263
:1006A000871D472A831687158312871D582B5C2BBD
:1006B000A70A0319A80A3D2A0A2A822B84011F309F
:1006C000830583169101073083129F00831605125C
:1006D000831205168316851583128519702B8F28B2
:1006E000831687168312871A762B3E2983160716E0
:1006F0008312071A7C2BC229831687158312871948
:10070000832B042A872B0A30AC00AD0057206A2BBC
:02071000630084
:02400E00043F6D
:00000001FF
